:100000008B1383160313FF30860010308500831294
:10001000031385018514051446204020061A1B2869
:10002000112818302520C8305E2046305E2006306A
:1000300025203A200B2813302520C8305E201930A7
:100040005E20063025203A200B288D003D20061921
:100050002728061D292885150000851100000000AD
:100060000000000000003A2028305A208D0B26287E
:100070003D200800051585100800851405110800AD
:10008000861940283D20861D43280800861A08004E
:100090003D20051C4C284E2805144F2805100D3016
:1000A0008F00FF308E00FF305A208E0B53288F0BAD
:1000B000512846288C008C0B5B2808008D000619FF
:1000C0005F28061D612828305A208D0B5F28080004
:02400E00FA3F77
:00000001FF
